:100000008316003086001F3085008312940195010D
:10001000960197018601051E1120851911204120A6
:100020000B28940A14080A3C03192C20051D1B20D8
:100030000519252008001930051C193E851C643E51
:1000400092004120920B212808004120051E2528FE
:1000500041208519282808009401950A15080A3CB2
:100060000319332008009501960A16080A3C031963
:100070003A2008009601970A17080A3C03199701CD
:100080000800013093001430840000088600131823
:1000900006169318861613190617931986175720F4
:1000A0008601931908000310930D840A4528033034
:1000B00090006E3091000000000000000000000081
:0C00C0000000910B5B28900B59280800F1
:00000001FF
